:100000000C9446000C9465000C9465000C946500FB
:100010000C9465000C9465000C9465000C946500CC
:100020000C9465000C9465000C9465000C946500BC
:100030000C9465000C9465000C9465000C946500AC
:100040000C9465000C9465000C9465000C9465009C
:100050000C9465000C9465000C9465000C9465008C
:100060000C9465000C9465000C9465000C9465007C
:100070000C9465000C9465000C9465000C9465006C
:100080000C9465000C9465000C94650011241FBE4F
:10009000CFEFD0E1DEBFCDBF12E0A0E0B1E0E4EDF4
:1000A000FFE100E00BBF02C007900D92AE32B10736
:1000B000D9F712E0AEE2B2E001C01D92A334B1075D
:1000C000E1F70E9465020C94E80F0C9400008DED9E
:1000D0008A95F1F70895929A9DED292F2A95F1F7C7
:1000E00088BB892F8A95F1F7949A892F8A95F1F721
:1000F00094989A95F1F7089592989DED292F2A9555
:10010000F1F788BB892F8A95F1F7949A892F8A9500
:10011000F1F794989A95F1F7089592989DED892FAB
:100120008A95F1F781E088BB892F8A95F1F7949A37
:10013000892F8A95F1F794989A95F1F7089518BA4E
:100140008FEF87BB12BA8CE381BB939894989298F7
:100150009DED892F8A95F1F78BE388BB892F8A95CE
:10016000F1F7949A892F8A95F1F79498892F8A95B7
:10017000F1F79298892F8A95F1F78CE088BB892F47
:100180008A95F1F7949A892F8A95F1F794989A9520
:10019000F1F70E948D000895823041F0833041F0E4
:1001A000813011F490E405C090E003C090E101C0FB
:1001B00090E5960F906892988DED282F2A95F1F78B
:1001C00098BB982F9A95F1F7949A982F9A95F1F7F2
:1001D00094988A95F1F70895FC012DED11C0929A3B
:1001E000822F8A95F1F798BB822F8A95F1F7949A1E
:1001F000822F8A95F1F79498822F8A95F1F731969C
:100200009081992361F70895FC012DED11C0929A18
:10021000822F8A95F1F798BB822F8A95F1F7949AED
:10022000822F8A95F1F79498822F8A95F1F731966B
:100230009081992361F70895382F6AE00E94A50FF5
:10024000805D929A2DED922F9A95F1F788BB822FBF
:100250008A95F1F7949A822F8A95F1F79498822FD4
:100260008A95F1F7832F0E94A50F905D929A822FB5
:100270008A95F1F798BB822F8A95F1F7949A822F8D
:100280008A95F1F794982A95F1F70895382F982FC9
:1002900092959F709A3010F4905D01C0995C929A8B
:1002A0008DED282F2A95F1F798BB982F9A95F1F7A5
:1002B000949A982F9A95F1F794988A95F1F7932F3D
:1002C0009F709A3010F4905D01C0995C929A8DED08
:1002D000282F2A95F1F798BB982F9A95F1F7949AC1
:1002E000982F9A95F1F794988A95F1F708951F93AE
:1002F000182F892F0E944601812F0E9446011F91CD
:10030000089522E08835920718F488E592E006C047
:1003100029E08136920710F080E699E0BC0180E088
:1003200090E00E94950A2AEF3DEE4BE65FE30E94C3
:10033000AF070E94D90570938700609386000895E7
:10034000853B910510F084EB90E0BC0133E0660F33
:10035000771F3A95E1F7880F991F680F791F685A40
:100360007D4F80E090E00E94950A2AEF3DEE4BE63B
:100370005FE30E94AF070E94D905709387006093E6
:10038000860008955F926F927F928F929F92AF92B4
:10039000BF92CF92DF92EF92FF920F931F93CF9372
:1003A000DF934C018D9AC0E0D0E050E2552E40E73B
:1003B000642E41E0742E75C082B3852582BBE2961F
:1003C000BE01882777FD8095982FE2970E94E30968
:1003D0005B016C0122E539E44DE950E40E94AF076E
:1003E0007B018C0120E030E040E85FE30E94B3092C
:1003F000882314F461E052C020E030E04FE753E47A
:10040000C801B7010E94530918160CF043C020E040
:1004100030E04AE754E4C601B5010E94A9085B0137
:100420006C0126E636E646E655E40E94AF077B01FE
:100430008C0120E030E040E85FE30E94B3098823AC
:100440001CF461E070E022C020E03FEF4FE757E48A
:10045000C801B7010E9453091816A4F420E030E047
:1004600040E251E4C601B5010E94AF070E94D905E0
:1004700005C0C3010197F1F7615070406115710526
:10048000C1F70EC0C801B7010E94D905CB01019781
:10049000F1F706C0C801B7010E94D9056A95F1F7C6
:1004A0002396C815D9050CF487CFDF91CF911F9102
:1004B0000F91FF90EF90DF90CF90BF90AF909F9003
:1004C0008F907F906F905F9008952F923F924F9200
:1004D0005F926F927F928F929F92AF92BF92CF92D4
:1004E000DF92EF92FF920F931F93DF93CF930F92C0
:1004F000CDB7DEB78FEF81BB14BA13B888E082B9ED
:1005000080E880938B0082E180938A0010928900BA
:100510001092880080E098E490938100809380009E
:10052000109287001092860010928500109284002D
:10053000109283001092820017BE10927D000E94DC
:100540009F000E948D008CEC9CE10197F1F72FEF4A
:100550002093220137B33983309342026091200106
:100560007091210180E090E00E94950A1B012C010E
:1005700022E539E44DE950E40E94AF075B016C01CC
:1005800020E030E040E85FE30E94B309882314F4E0
:1005900061E053C020E030E04FE753E4C601B5010D
:1005A0000E94530918160CF044C020E030E04AE7DE
:1005B00054E4C201B1010E94A9083B014C0126E6A6
:1005C00036E646E655E40E94AF077B018C0120E049
:1005D00030E040E85FE30E94B30988231CF461E047
:1005E00070E023C020E03FEF4FE757E4C801B701B8
:1005F0000E9453091816ACF420E030E040E251E4C8
:10060000C401B3010E94AF070E94D90506C080E76C
:1006100091E00197F1F76150704061157105B9F7EC
:100620000EC0C801B7010E94D905CB010197F1F7AF
:1006300006C0C601B5010E94D9056A95F1F7B89ABE
:10064000B99ABA9ABB9ABC98BD98BE98BF988EE0EA
:1006500088BB20E030E040E85FE3C601B5010E94BE
:10066000B309882314F461E053C020E030E04FE781
:1006700053E4C601B5010E94530918160CF044C09A
:1006800020E030E04AE754E4C201B1010E94A90829
:100690003B014C0126E636E646E655E40E94AF07EC
:1006A0007B018C0120E030E040E85FE30E94B30969
:1006B00088231CF461E070E023C020E03FEF4FE7A7
:1006C00057E4C801B7010E9453091816ACF420E0A2
:1006D00030E040E251E4C401B3010E94AF070E9440
:1006E000D90506C080E791E00197F1F761507040AD
:1006F00061157105B9F70EC0C801B7010E94D9058F
:10070000CB010197F1F706C0C601B5010E94D905DA
:100710006A95F1F7B49903C091E090932201B599DD
:1007200003C0E4E0E0932201B69903C0F7E0F09340
:100730002201B79903C024E6209322013DE038BB93
:1007400020E030E040E85FE3C601B5010E94B30954
:10075000882314F461E053C020E030E04FE753E415
:10076000C601B5010E94530918160CF044C020E0E0
:1007700030E04AE754E4C201B1010E94A9083B01FC
:100780004C0126E636E646E655E40E94AF077B01BB
:100790008C0120E030E040E85FE30E94B309882349
:1007A0001CF461E070E023C020E03FEF4FE757E426
:1007B000C801B7010E9453091816ACF420E030E0DC
:1007C00040E251E4C401B3010E94AF070E94D90581
:1007D00006C080E791E00197F1F761507040611524
:1007E0007105B9F70EC0C801B7010E94D905CB0148
:1007F0000197F1F706C0C601B5010E94D9056A95B7
:10080000F1F7B49903C082E080932201B59903C047
:1008100095E090932201B69903C0E8E0E0932201AD
:10082000B79902C010922201FBE0F8BB20E030E053
:1008300040E85FE3C601B5010E94B309882314F4C0
:1008400061E053C020E030E04FE753E4C601B5015A
:100850000E94530918160CF044C020E030E04AE72B
:1008600054E4C201B1010E94A9083B014C0126E6F3
:1008700036E646E655E40E94AF077B018C0120E096
:1008800030E040E85FE30E94B30988231CF461E094
:1008900070E023C020E03FEF4FE757E4C801B70105
:1008A0000E9453091816ACF420E030E040E251E415
:1008B000C401B3010E94AF070E94D90506C080E7BA
:1008C00091E00197F1F76150704061157105B9F73A
:1008D0000EC0C801B7010E94D905CB010197F1F7FD
:1008E00006C0C601B5010E94D9056A95F1F7B49911
:1008F00003C023E020932201B59903C036E0309372
:100900002201B69903C089E080932201B79903C000
:1009100085E68093220197E098BB20E030E040E834
:100920005FE3C601B5010E94B309882314F461E0B6
:1009300053C020E030E04FE753E4C601B5010E9408
:10094000530918160CF044C020E030E04AE754E4A4
:10095000C201B1010E94A9085B016C0126E636E6DE
:1009600046E655E40E94AF077B018C0120E030E0B1
:1009700040E85FE30E94B30988231CF461E070E063
:1009800023C020E03FEF4FE757E4C801B7010E94C2
:1009900053091816ACF420E030E040E251E4C601FF
:1009A000B5010E94AF070E94D90506C080E791E01B
:1009B0000197F1F76150704061157105B9F70EC0EC
:1009C000C801B7010E94D905CB010197F1F706C014
:1009D000C601B5010E94D9056A95F1F7B49903C023
:1009E000EBE0E0932201B59903C08CE080932201F3
:1009F000B69903C0FDE0F0932201B79903C02EE041
:100A0000209322018FE088BB8F9A82B3805882BBEB
:100A1000398137BB9091220180912301981709F405
:100A20007BC090932301963041F480912401843B54
:100A300079F18A3A68F5865F22C0943041F480915A
:100A40002401882329F18B3018F18A5018C099307D
:100A500031F480912401843BD9F08E5F10C097302F
:100A600031F480912401882399F0825008C092309B
:100A700019F4109224010CC0983021F484EB809377
:100A8000240106C0953021F480ED97E00E94C20158
:100A900080912301882309F03FC088E292E090937F
:100AA00087008093860080E197E2E0E7F1E03197EC
:100AB000F1F70197D1F71092240127C09AE0899F9E
:100AC000B0011124685A7D4F80E090E00E94950AA1
:100AD0002AEF3DEE4BE65FE30E94AF070E94D90587
:100AE000709387006093860088EE93E0E0E7F1E082
:100AF0003197F1F70197D1F788EE93E00E94C20198
:100B000080912401865F8093240180912401853B9C
:100B1000A8F28AE58093240160E080E00E94CC0086
:100B200080E091E00E94EC0060E081E00E94CC0057
:100B30008091240190E09F938F93E0E1F1E0FF9397
:100B4000EF932EE232E03F932F930E94030D8EE24B
:100B500092E00E94EC002091240130E0C901EDB741
:100B6000FEB736960FB6F894FEBF0FBEEDBF853BBD
:100B7000910510F084EB90E0BC01F3E0660F771F65
:100B8000FA95E1F7880F991F680F791F685A7D4F12
:100B900080E090E00E94950A2AEF3DEE4BE65FE38D
:100BA0000E94AF070E94D90570938700609386006A
:100BB000CECCEF92FF920F931F937B018C0120E02C
:100BC00030E040E05FE40E94830988238CF020E05D
:100BD00030E040E05FE4C801B7010E9451070E9485
:100BE000410A9B01AC01205030404040504806C0B3
:100BF000C801B7010E94410A9B01AC01B901CA01B9
:100C00001F910F91FF90EF900895A0E0B0E0EBE00E
:100C1000F6E00C94B10FDC012B01FA019C919230AB
:100C200008F439C1EB018881823008F433C1943073
:100C300069F4843009F02FC111969C911197898134
:100C4000981709F428C1A5E2B1E025C1843009F460
:100C500021C18230A9F4923009F01DC19A01AD0181
:100C600088E0EA010990AE01E90109929E018150F4
:100C7000C1F7E201898111969C918923818308C182
:100C8000923009F407C112962D903C901397EB0116
:100C90008A819B811496AD90BD90CD90DC90179782
:100CA000EC80FD800E811F819101281B390BB90159
:100CB00037FF04C066277727621B730B603271050C
:100CC0000CF061C0121613066CF537014801062EB0
:100CD00004C096948794779467940A94D2F721E09D
:100CE00030E040E050E004C0220F331F441F551F86
:100CF0006A95D2F721503040404050402E213F218C
:100D000040235123211531054105510521F021E0F2
:100D100030E040E050E079018A01E628F728082910
:100D200019293CC0232BD1F1260E371E350146016F
:100D3000062E04C096948794779467940A94D2F709
:100D400021E030E040E050E004C0220F331F441F98
:100D5000551F6A95D2F721503040404050402A211B
:100D60003B214C215D21211531054105510521F023
:100D700021E030E040E050E059016A01A628B728A0
:100D8000C828D9280BC0821593052CF01C01AA2471
:100D9000BB24650103C0EE24FF24870111969C91BA
:100DA000D20111968C91981709F445C0992339F016
:100DB000A80197012A193B094C095D0906C0A60143
:100DC00095012E193F09400B510B57FD08C01182A8
:100DD0003382228224833583468357831DC081E07A
:100DE00081833382228288279927DC01821B930B1F
:100DF000A40BB50B84839583A683B7830DC0220F04
:100E0000331F441F551F24833583468357838281B4
:100E10009381019793838283248135814681578111
:100E2000DA01C9010197A109B1098F5F9F4FAF4F47
:100E3000BF4328F30BC0918333822282EA0CFB1C50
:100E40000C1D1D1DE482F5820683178383E08083D9
:100E5000248135814681578157FF1AC0C901AA27CD
:100E600097FDA095BA2F81709070A070B0705695C4
:100E7000479537952795822B932BA42BB52B8483ED
:100E80009583A683B783828193810196938382831E
:100E9000DF0101C0D201CD01CDB7DEB7E2E10C9494
:100EA000CD0FA0E2B0E0E7E5F7E00C94BD0F698359
:100EB0007A838B839C832D833E834F835887E9E01D
:100EC000EE2EF12CEC0EFD1EB701CE0101960E9414
:100ED000320C8E010F5E1F4FB801CE0105960E94A5
:100EE000320C8A8991E089278A8BAE01475E5F4F79
:100EF000B801C7010E9405060E945D0BA096E6E0BE
:100F00000C94D90FA0E2B0E0E8E8F7E00C94BD0F34
:100F100069837A838B839C832D833E834F83588799
:100F2000F9E0EF2EF12CEC0EFD1EB701CE0101967B
:100F30000E94320C8E010F5E1F4FB801CE01059644
:100F40000E94320CAE01475E5F4FB801C7010E949C
:100F500005060E945D0BA096E6E00C94D90FA0E276
:100F6000B0E0E5EBF7E00C94B10F69837A838B83F3
:100F70009C832D833E834F835887BE01675F7F4FDD
:100F8000CE0101960E94320CBE016F5E7F4FCE01F2
:100F900005960E94320C9985923088F089898230BA
:100FA000C8F0943019F4823051F404C0843029F42C
:100FB000923081F485E291E0C6C0923049F420E09D
:100FC0009A858A89981321E02A87CE010996BBC0A9
:100FD000823049F420E09A858A89981321E02A8B8F
:100FE000CE014196B0C02D843E844F8458886D88D0
:100FF0007E888F88988CEE24FF248701AA24BB2446
:10100000650140E050E060E070E0E0E0F0E0C10148
:1010100081709070892BE9F0E60CF71C081D191DF2
:101020009A01AB012A0D3B1D4C1D5D1D80E090E037
:10103000A0E0B0E0E614F7040805190520F481E00B
:1010400090E0A0E0B0E0BA01A901480F591F6A1F63
:101050007B1FAA0CBB1CCC1CDD1C97FE08C081E0CA
:1010600090E0A0E0B0E0A82AB92ACA2ADB2A31968B
:10107000E032F10549F0660C771C881C991C5694E7
:10108000479437942794C3CFFA85EA892B893C8902
:101090008B859C85280F391F2E5F3F4F17C0CA01D3
:1010A00081709070892B61F016950795F794E794FD
:1010B00080E090E0A0E0B0E8E82AF92A0A2B1B2B98
:1010C00076956795579547952F5F3F4F77FDE7CF0B
:1010D0000CC0440F551F661F771F17FD4160EE0CB3
:1010E000FF1C001F111F21503040403090E0590775
:1010F00090E0690790E4790760F32B8F3C8FDB0168
:10110000CA018F779070A070B07080349105A105EE
:10111000B10561F447FD0AC0E114F10401051105B0
:1011200029F0405C5F4F6F4F7F4F40781A8EFE175B
:1011300011F081E08A8F4D8F5E8F6F8F78A383E0EF
:10114000898FCE0149960E945D0BA096E2E10C9436
:10115000CD0FA8E1B0E0EFEAF8E00C94B90F698395
:101160007A838B839C832D833E834F835887B9E09A
:10117000EB2EF12CEC0EFD1EB701CE0101960E9464
:10118000320C8E010F5E1F4FB801CE0105960E94F2
:10119000320C2985223008F47CC03989323010F4B1
:1011A000B8017AC08A859A8989278A87243011F004
:1011B000223031F4231709F06CC065E271E06CC095
:1011C000343039F41D861E861F86188A1C861B86BD
:1011D00004C0323021F484E08987B7015DC02B85DB
:1011E0003C858B899C89281B390B3C872B87ED8498
:1011F000FE840F851889AD88BE88CF88D88CEA1404
:10120000FB040C051D0540F4EE0CFF1C001F111F14
:10121000215030403C872B8720E030E040E050E018
:1012200080E090E0A0E0B0E46FE170E0EA14FB043D
:101230000C051D0540F0282B392B4A2B5B2BEA1897
:10124000FB080C091D09B695A79597958795EE0C97
:10125000FF1C001F111F6150704041F7DA01C901E6
:101260008F779070A070B07080349105A105B105A2
:1012700061F427FD0AC0E114F1040105110529F00C
:10128000205C3F4F4F4F5F4F20782D873E874F8721
:10129000588BBE01675F7F4FCB010E945D0B689644
:1012A000EAE00C94D50FA8E1B0E0E9E5F9E00C9490
:1012B000BD0F69837A838B839C832D833E834F8309
:1012C000588789E0E82EF12CEC0EFD1EB701CE0107
:1012D00001960E94320C8E010F5E1F4FB801CE01A5
:1012E00005960E94320C8985823040F089898230CF
:1012F00028F0B801C7010E94AA0C01C08FEF6896C0
:10130000E6E00C94D90FA8E1B0E0E9E8F9E00C942C
:10131000BD0F69837A838B839C832D833E834F83A8
:10132000588789E0E82EF12CEC0EFD1EB701CE01A6
:1013300001960E94320C8E010F5E1F4FB801CE0144
:1013400005960E94320C8985823040F0898982306E
:1013500028F0B801C7010E94AA0C01C08FEF68965F
:10136000E6E00C94D90FA8E1B0E0E9EBF9E00C94C9
:10137000BD0F69837A838B839C832D833E834F8348
:10138000588789E0E82EF12CEC0EFD1EB701CE0146
:1013900001960E94320C8E010F5E1F4FB801CE01E4
:1013A00005960E94320C8985823040F0898982300E
:1013B00028F0B801C7010E94AA0C01C081E068961C
:1013C000E6E00C94D90FA8E0B0E0E9EEF9E00C9467
:1013D000BA0F9B01AC0183E08983DA01C901882738
:1013E000B7FD83959927AA27BB27B82E211531056C
:1013F0004105510519F482E089833AC08823A9F098
:10140000203080E0380780E0480780E8580729F45A
:1014100060E070E080E09FEC30C0EE24FF248701A4
:10142000E21AF30A040B150B02C079018A018EE15E
:10143000C82ED12CDC82CB82ED82FE820F831887EE
:10144000C801B7010E940E0B01971816190684F403
:10145000082E04C0EE0CFF1C001F111F0A94D2F7C7
:10146000ED82FE820F831887C81AD90ADC82CB82EC
:10147000BA82CE0101960E945D0B2896E9E00C9499
:10148000D60FACE0B0E0E7E4FAE00C94C10F69835A
:101490007A838B839C83BE016B5F7F4FCE01019665
:1014A0000E94320C8D81823061F1823050F18430A3
:1014B00021F48E81882351F12EC02F81388537FD8C
:1014C00020C06E812F3131051CF06623F9F023C056
:1014D0008EE190E0821B930B29853A854B855C85D4
:1014E00004C056954795379527958A95D2F7662378
:1014F000B1F050954095309521953F4F4F4F5F4F3C
:101500000EC020E030E040E050E009C02FEF3FEF98
:101510004FEF5FE704C020E030E040E050E8B90161
:10152000CA012C96E2E00C94DD0FA8E0B0E0EBE9F4
:10153000FAE00C94BB0F7B018C01611571058105EC
:10154000910519F482E0898360C083E089838EE18C
:10155000C82ED12CDC82CB82ED82FE820F831887CD
:10156000C801B7010E940E0BBC016150704077FFAB
:1015700039C0EE27FF27E61BF70B20E030E040E004
:1015800050E081E090E0A0E0B0E00E2E04C0880FB3
:10159000991FAA1FBB1F0A94D2F70197A109B1098D
:1015A0008E219F21A023B1230097A105B10521F031
:1015B00021E030E040E050E004C016950795F79434
:1015C000E794EA95D2F72E293F29402B512B2D8302
:1015D0003E834F8358878EE190E0861B970B9C8358
:1015E0008B8313C06115710581F0062E04C0EE0CCB
:1015F000FF1C001F111F0A94D2F7ED82FE820F8399
:101600001887C61AD70ADC82CB821A82CE010196CD
:101610000E945D0B2896E8E00C94D70FEF92FF92A2
:101620000F931F937B018C0180E0E81680E0F806A1
:1016300081E0080780E0180788F48FEFE816F104CE
:101640000105110531F028F088E090E0A0E0B0E05D
:1016500017C080E090E0A0E0B0E012C080E0E816A3
:1016600080E0F80680E0080781E0180728F088E1AC
:1016700090E0A0E0B0E004C080E190E0A0E0B0E045
:1016800020E230E040E050E0281B390B4A0B5B0BB6
:1016900004C016950795F794E7948A95D2F7F70159
:1016A000E35DFE4F8081281B310941095109C901C1
:1016B0001F910F91FF90EF900895DF92EF92FF92AC
:1016C0000F931F93FC01E480F58006811781D18080
:1016D0008081823048F480E090E0A0E1B0E0E82A28
:1016E000F92A0A2B1B2BA5C0843009F49FC0823035
:1016F00021F4EE24FF24870105C0E114F104010563
:10170000110519F4E0E0F0E096C0628173819FEF6B
:10171000623879070CF05BC022E83FEF261B370BDD
:101720002A3131052CF020E030E040E050E02AC0C2
:10173000B801A701022E04C0769567955795479585
:101740000A94D2F781E090E0A0E0B0E004C0880FF6
:10175000991FAA1FBB1F2A95D2F70197A109B109AA
:101760008E219F21A023B1230097A105B10521F06F
:1017700081E090E0A0E0B0E09A01AB01282B392B8A
:101780004A2B5B2BDA01C9018F779070A070B07083
:1017900080349105A105B10539F427FF09C0205C0B
:1017A0003F4F4F4F5F4F04C0215C3F4F4F4F5F4F44
:1017B000E0E0F0E02030A0E03A07A0E04A07A0E433
:1017C0005A0710F0E1E0F0E079018A0127C06038A3
:1017D000710564F5FB01E158FF4FD801C7018F7710
:1017E0009070A070B07080349105A105B10539F4F6
:1017F000E7FE0DC080E490E0A0E0B0E004C08FE31D
:1018000090E0A0E0B0E0E80EF91E0A1F1B1F17FFD2
:1018100005C016950795F794E794319687E01695DD
:101820000795F794E7948A95D1F705C0EE24FF2435
:101830008701EFEFF0E06E2F679566276795902F91
:101840009F77D794DD24D7948E2F8695492F462BEA
:10185000582F5D29B701CA011F910F91FF90EF909A
:10186000DF900895FC01DB01408151812281622FCC
:101870006F7770E0221F2227221F9381892F880F04
:10188000822B282F30E0991F9927991F11969C933E
:10189000119721153105A9F541155105610571050E
:1018A00011F482E037C082E89FEF13969C938E93E9
:1018B00012979A01AB0167E0220F331F441F551F97
:1018C0006A95D1F783E08C930DC0220F331F441F1C
:1018D000551F12968D919C911397019713969C9387
:1018E0008E931297203080E0380780E0480780E42C
:1018F000580758F314962D933D934D935C93179787
:1019000008952F3F310579F44115510561057105A1
:1019100019F484E08C93089564FF03C081E08C93F4
:1019200012C01C9210C02F57304013963C932E9338
:10193000129783E08C9387E0440F551F661F771F33
:101940008A95D1F7706414964D935D936D937C9353
:10195000179708951F93DC01FB019C91923008F4C6
:1019600047C08081823008F443C0943051F411960E
:101970001C91843099F58181682F70E0611B710999
:101980003FC0843021F0923031F48230B9F181814E
:10199000882389F12DC011961C9111978230F1F0A6
:1019A00081811817D9F412962D913C911397828159
:1019B00093818217930794F028173907BCF0149687
:1019C0008D919D910D90BC91A02D248135814681F2
:1019D0005781281739074A075B0718F4112341F08C
:1019E0000AC082179307A407B50740F4112319F022
:1019F00061E070E005C06FEF7FEF02C060E070E073
:101A0000CB011F910895AEE0B0E0E9E0FDE00C9459
:101A1000BF0F0D891E8986E08C831A8309838FEF9F
:101A20009FE79E838D83CE014996AC016F89788DA7
:101A3000CE0101960E94260D2F813885020F131FBB
:101A4000F80110822E96E4E00C94DB0FABE0B0E0DE
:101A5000ECE2FDE00C94B10F3C012B015A01FC01BA
:101A600017821682838181FD03C06FEF7FEFC8C1AB
:101A70009AE0892E1E010894211C311CF301238158
:101A8000F20123FD859123FF81912F01882309F421
:101A9000B4C1853239F423FD859123FF81912F0153
:101AA000853229F4B30190E00E941B0FE7CF982FF5
:101AB000DD24CC249924FFE1FD15D0F09B3269F0A0
:101AC0009C3228F4903259F0933291F40EC09D323A
:101AD00049F0903369F441E024C052E0D52A84E013
:101AE000D82A28C098E0D92A25C0E0E1DE2A22C001
:101AF000D7FC29C0892F80538A3070F4D6FE05C0E8
:101B0000989C902C1124980E15C0C89CC02C1124B0
:101B1000C80EF0E2DF2A0EC09E3229F4D6FC6DC159
:101B200040E4D42A07C09C3619F450E8D52A02C0F4
:101B3000983649F4F20123FD959123FF91912F01ED
:101B4000992309F0B8CF892F8554833018F080523B
:101B5000833038F444E050E0A40EB51E5FE35983AF
:101B60000FC0933631F0933779F0933509F056C0B2
:101B700020C0F5018081898342E050E0A40EB51EAB
:101B8000710101E010E012C0F501E080F180D6FCA7
:101B900003C06FEF7FEF02C0692D70E042E050E0BC
:101BA000A40EB51EC7010E94100F8C015FE7D5225D
:101BB00014C0F501E080F180D6FC03C06FEF7FEF29
:101BC00002C0692D70E042E050E0A40EB51EC701CE
:101BD0000E94050F8C0150E8D52AD3FE07C01AC019
:101BE000B30180E290E00E941B0FCA948C2D90E01C
:101BF00008171907A8F30EC0F701D7FC8591D7FE87
:101C000081917F01B30190E00E941B0FC110CA9423
:101C1000015010400115110579F7ECC0943611F010
:101C2000993671F5D7FE08C0F501E080F180028198
:101C3000138144E050E00AC0F501808191817C016C
:101C40000027F7FC0095102F42E050E0A40EB51ECF
:101C50005FE6D52217FF0AC010950095F094E09436
:101C6000E11CF11C011D111D80E8D82A2AE030E09A
:101C7000A101C801B7010E94470FF82EF21840C019
:101C8000953729F41D2D1F7E2AE030E01DC01D2D43
:101C9000197F9F3661F0903720F4983509F0ADC078
:101CA0000FC0903739F0983709F0A7C004C028E07A
:101CB00030E00AC0106114FD146020E130E004C07F
:101CC00014FD166020E132E017FF08C0F5016081C5
:101CD00071818281938144E050E008C0F5018081E8
:101CE0009181BC0180E090E042E050E0A40EB51E7E
:101CF000A1010E94470FF82EF2188FE7D82ED122AB
:101D0000D6FE0BC05EEFD522F91438F4D4FE07C01E
:101D1000D2FC05C08FEED82202C01F2D01C0192DA4
:101D2000D4FE0DC0FE01EF0DF11D8081803319F44A
:101D300099EED92208C01F5FD2FE05C003C08D2DC9
:101D4000867809F01F5F0D2DD3FC14C0D0FE0FC0A4
:101D50001C1510F09F2C0BC09F2C9C0C911A1C2D55
:101D600006C0B30180E290E00E941B0F1F5F1C15AC
:101D7000C0F304C01C1510F4C11A01C0CC2404FF28
:101D800010C0B30180E390E00E941B0F02FF1EC051
:101D900001FD03C088E790E002C088E590E0B30150
:101DA0000CC0802F867891F001FF02C08BE201C049
:101DB00080E2D7FC8DE2B30190E00E941B0F06C0C9
:101DC000B30180E390E00E941B0F9A94F914C0F3D2
:101DD000FA94F101EF0DF11DB301808190E00E94B2
:101DE0001B0FFF20A9F706C0B30180E290E00E941C
:101DF0001B0FCA94CC20C1F741CEF30166817781D5
:101E0000CB012B96E2E10C94CD0FFC0105906150C3
:101E100070400110D8F7809590958E0F9F1F089500
:101E2000FC016150704001900110D8F780959095A9
:101E30008E0F9F1F08950F931F93CF93DF938C01F5
:101E4000EB018B8181FF1BC082FF0DC02E813F8182
:101E50008C819D812817390764F4E881F981019309
:101E6000F983E88306C0E885F985802F0995892BD9
:101E700031F48E819F8101969F838E8302C00FEF84
:101E80001FEFC801DF91CF911F910F910895FA01C3
:101E9000AA27283051F1203181F1E8946F936E7FA9
:101EA0006E5F7F4F8F4F9F4FAF4FB1E03ED0B4E09A
:101EB0003CD0670F781F891F9A1FA11D680F791FDB
:101EC0008A1F911DA11D6A0F711D811D911DA11DEC
:101ED00020D009F468943F912AE0269F11243019FC
:101EE000305D3193DEF6CF010895462F4770405D97
:101EF0004193B3E00FD0C9F7F6CF462F4F70405D46
:101F00004A3318F0495D31FD4052419302D0A9F7A0
:101F1000EACFB4E0A6959795879577956795BA959A
:101F2000C9F700976105710508959B01AC010A2E60
:101F300006945795479537952795BA95C9F7620F37
:101F4000731F841F951FA01D0895991B79E004C07D
:101F5000991F961708F0961B881F7A95C9F78095E8
:101F600008952F923F924F925F926F927F928F923D
:101F70009F92AF92BF92CF92DF92EF92FF920F9318
:101F80001F93CF93DF93CDB7DEB7CA1BDB0B0FB622
:101F9000F894DEBF0FBECDBF09942A8839884888DF
:101FA0005F846E847D848C849B84AA84B984C88475
:101FB000DF80EE80FD800C811B81AA81B981CE0F6C
:101FC000D11D0FB6F894DEBF0FBECDBFED01089551
:041FD000F894FFCFB3
:101FD4005679737475702050574D3A20504533002C
:101FE4002020205568656C3D202533642020200086
:101FF4000A00FFFF5A000000000000000000010278
:10200400020303030304040404040404040505058F
:102014000505050505050505050505050506060669
:10202400060606060606060606060606060606064C
:102034000606060606060606060606060607070739
:10204400070707070707070707070707070707071C
:10205400070707070707070707070707070707070C
:1020640007070707070707070707070707070707FC
:1020740007070707070707070707070707080808E9
:1020840008080808080808080808080808080808CC
:1020940008080808080808080808080808080808BC
:1020A40008080808080808080808080808080808AC
:1020B400080808080808080808080808080808089C
:1020C400080808080808080808080808080808088C
:1020D400080808080808080808080808080808087C
:1020E400080808080808080808080808080808086C
:0E20F400080808080808080808080808080076
:00000001FF
